:100AE800696E71756972650073706565643A25642D
:100AF800206D2F6D696E206D696C656167653A259B
:100B080064206D0D0A006D6F64656C004D6F64653F
:100B18006C20534554204F4B0D0A00636C6561727D
:100B2800007265736574206D696C65616765204F37
:100B38004B210D0A007370656564007365743A0093
:100B480028002C0029005573657220534554204F06
:050B58004B210D0A0015
:0F0CC80002230000012600012500C109012200BE
:100E37007C64EF4E60131CEC60087D0A1DED60F6C4
:090E470080FAEF1F70EC1E80E937
:010E5000227F
:100E9B00758921759850758DFD858D8BE4F587D2FD
:060EAB00AFD2ACD28E2292
:07000300AE071FEE70FA22A8
:0E0ED400C2ACC2998F993099FDC299D2AC225E
:100E83001207D3FF6011120ED47F05120003740101
:080E930029F9E43AFA80E92292
:100C9100E4FEAD517F03120E6A7F027E00120E3711
:100CA100E552FF3395E0FEAD077F05120E6A7F0224
:100CB1007E00120E377E00AF53AD077F06120E6A1B
:070CC1007F027E00020E37E6
:10038200E4F556F557F558F559F55AF55B2009038A
:1003920002060D755FFF75600A7561E8FB7A0079E8
:1003A20028120A66E94A4B60367E007F287D007B70
:1003B200007A007928120889755FFF75600A7561F5
:1003C200F0850A62850B638510648511657B007A6E
:1003D2000079281200827B007A0079280204627573
:1003E2005FFF75600B75610E7B007A007928120A37
:1003F20066E94A4B6048E52570057525018003E4EE
:10040200F525E5257004F523F5247E007F287D007F
:100412007B007A007928120889755FFF75600B7579
:1004220061147B007A0079281200827B007A0079BD
:1004320028120E83AD257F04120E6A0205FC755F39
:10044200FF75600B7561237B007A007928120A66BA
:10045200E94A4B6011E4F510F5117BFF7A0B79291B
:10046200120E830205FC755FFF75600B75613D7BA3
:10047200007A007928120A66E94A4B601F0524E5D2
:100482002470020523C39404E52394004005E4F597
:1004920023F5248523508524510205FC755FFF75E1
:1004A200600B7561437B007A007928120A66E94A7B
:1004B2004B70030205FC755FFF75600B7561487B2D
:1004C200007A007928120A66AE02C3E99428F55729
:1004D200EE9400F556755FFF75600B75614A7B00FF
:1004E2007A007928120A66AE02C3E99428F559EE19
:1004F2009400F558E4F550F551E5572401F55BE415
:100502003556F55AC3E55B9559E5586480F8E55AC6
:10051200648098502A7428255BF8E624D0FBE434E2
:10052200FFFAAE50AF517C007D0A1207ECEF2BF5BB
:1005320051EE3AF550055BE55B70C9055A80C5D3AB
:10054200E5519401E5506480948040067550007531
:100552005101755FFF75600B75614A7B007A007906
:1005620028120A66AE02C3E99428F557EE9400F504
:1005720056755FFF75600B75614C7B007A007928B8
:10058200120A66AE02C3E99428F559EE9400F558B2
:10059200E4F552F553E5572401F55BE43556F55A77
:1005A200C3E55B9559E5586480F8E55A6480985034
:1005B2002A7428255BF8E624D0FBE434FFFAAE5215
:1005C200AF537C007D0A1207ECEF2BF553EE3AF5A0
:1005D20052055BE55B70C9055A80C5D3E551940F9E
:1005E200E550648094A7400675502775510F7BFF34
:1005F2007A0B794E120E83120C917E007F287D00B9
:0B0602007B007A007928120889C209E9
:01060D0022CA
:100BC0007F01120D98EF75F0FFA4FFAEF0C006C0D4
:100BD000077F02120D98EFFDD0E02DF511D0E03423
:100BE00000F5107F03120D987550008F517F04128D
:100BF0000D988F257F05120D98EF75F0FFA4FFAEBD
:100C0000F0C006C0077F06120D98EFFDD0E02DF56D
:080C100053D0E03400F552223C
:100DFB00E5107E00FD7F01120E6A7FC81200037E94
:0F0E0B0000AF11AD077F02120E6A7FC80200030D
:100E1A00120E51120EB1120E9B120BC0120B5D1262
:0D0E2A00060E120D24120382120DFB80EF44
:03002300020C5973
:090C5900C0E0C0D075D000C0005D
:100C6200200925309820C29885992774282522F8D2
:100C7200A62774282522F8E6B40D07752200D209AA
:080C8200800605228002C299E0
:070C8A00D000D0D0D0E03211
:100CFA00C2958FA07F017E00120D0BD2947F057ED4
:010D0A0000E8
:100D0B00D3EF9400EE9400400F7DC77C01DCFEDD39
:080D1B00FAEF1F70EB1E80E8E7
:010D230022AD
:0A0EFB00C294C296120CFAC29422AF
:0A0F0500C294D296120CFAC2942294
:100E51007F38120EFB7F0C120EFB7F06120EFB7FFA
:090E610001120EFB7F80020EFB62
:0B0CD700011500011400011300C10A08
:100DDB00E4FDFCC3ED9FEC9E5015E4FBFA0BBB004E
:0F0DEB00010ABA07F8BBD0F50DBD00010C80E47A
:010DFA0022D6
:100B5D00E525602B855023855124C3E5539511F56B
:100B6D0055E5529510F554C3648094805005E4F515
:100B7D0054F555E5554554700BF523F5248005E4E2
:100B8D00F554F555E52445237004F513801DE52432
:100B9D006401452370057513028010E52464024538
:100BAD002370057513058003751307851314C29201
:030BBD00D29322AE
:100DBA000515A20AB35017E51595145004D2978069
:100DCA0002C297E515C394144006E4F51522C297AA
:010DDA0022F6
:050EE200120EE7D291A1
:080EE7007F017E02DEFEDFFA4E
:010EEF0022E0
:0F0EC500D290120EE2C290120EE7C291020EE717
:0A0F0F00C290120EE2D290020EE72B
:020C1800AD0726
:100C1A00E4FBFAEDC4131313540124FF9290ED255B
:100C2A00E0FD120EE2C291120EE70BBB08E5D2906C
:100C3A00120EE7D29130900F0AEAD394C840F6C256
:0E0C4A0091120EE77F0022C291120EE77F0189
:010C58002279
:100D7200E4FDFCD290120EE7D291120EE7EC25E0D0
:100D8200FCA290E4334204120EE7C291120EE70D68
:050D9200BD08E5AF04FF
:010D97002239
:100E6A00AC05A907120EC57FA0120C18AF01120C0F
:090E7A0018AF04120C18020F0F4E
:020D9800AC07A6
:100D9A00120EC57FA0120C18AF04120C18120EC541
:0F0DAA007FA1120C18120D72AD07120F0FAF05BB
:010DB9002217
:100CE20002100000020C0000011200020A000002C1
:070CF2000E000002080000E3
:0B0EF000EF1FAC0670011E4C70F622D4
:100EB100758921758CFC758A18D2A9D28CD2AFD2D2
:040EC100AAD28A2205
:10060E007F82120EFBAE0AAF0B7C007D641207FEDA
:10061E007C007D0A1207FEED2430FF120F05AE0A94
:10062E00AF0B7C007D0A1207FE7C007D0A1207FECE
:10063E00ED2430FF120F05AE0AAF0B7C007D0A12BF
:10064E0007FEED2430FF120F057F88120EFBAE1051
:10065E00AF117C037DE81207FE7C007D0A1207FEB7
:10066E00ED2430FF120F05AE10AF117C007D641229
:10067E0007FE7C007D0A1207FEED2430FF120F05E7
:10068E00AE10AF117C007D0A1207FE7C007D0A12AF
:10069E0007FEED2430FF120F05AE10AF117C007D6A
:1006AE000A1207FEED2430FF120F057F6D120F05A3
:1006BE007F8E120EFBE524452370047F4E8022E5CB
:1006CE00246401452370047F4C8016E524640245A2
:1006DE002370047F4D800AE5246403452370057F53
:1006EE0048120F057FC0120EFBAE52AF537C037D36
:1006FE00E81208537C007D0A120853ED2430FF12D5
:10070E000F05AE52AF537C007D641208537C007D02
:10071E000A120853ED2430FF120F05AE52AF537C70
:10072E00007D0A1208537C007D0A120853ED243016
:10073E00FF120F05AE52AF537C007D0A120853ED27
:10074E002430FF120F057F6D120F057FC8120EFBAE
:10075E00AE54AF557C037DE81208537C007D0A121F
:10076E000853ED2430FF120F05AE54AF557C007DBB
:10077E00641208537C007D0A120853ED2430FF12D8
:10078E000F05AE54AF557C007D0A1208537C007DD8
:10079E000A120853ED2430FF120F05AE54AF557CEC
:1007AE00007D0A120853ED2430FF120F057F6D12E3
:1007BE000F057FCE120EFBE52570047F4480027F6D
:0507CE0053120F05228B
:100D240020B5237FE87E03120EF020B5160524E5D6
:100D34002470020523C39404E52394004005E4F5DC
:070D440023F52430B5FD2268
:03000B0002092ABD
:10092A00C0E0C0F0C083C082C0D075D000C000C093
:0D093A0001C002C003C004C005C006C00714
:10094700758CFC758A180509E50970020508120DF2
:10095700BAC3E50994F4E50864809481405AC2AAB1
:10096700750800750900AE0CAF0D7C007D031207FA
:10097700EC7D141207FE8E0E8F0F7C007D0C120784
:10098700EC8E0A8F0BAE0CAF0D7D141207FE7C00A8
:100997007D031207ECEF2511F511EE3510F510D395
:1009A700E511940FE5109427400675102775110F70
:0809B700750C00750D00D2AAB9
:1009BF00D007D006D005D004D003D002D001D0008C
:0B09CF00D0D0D082D083D0F0D0E03236
:03001300020016D2
:0D001600C0E0050DE50D7002050CD0E032D4
:030000000209DA18
:0C09DA00787FE4F6D8FD75816F020A21D9
:1007D300BB010689828A83E0225002E722BBFE0224
:0907E300E32289828A83E4932257
:1007EC00EF8DF0A4A8F0CF8CF0A428CE8DF0A42E21
:0207FC00FE22DB
:1007FE00BC000BBE0029EF8DF084FFADF022E4CCDF
:10080E00F875F008EF2FFFEE33FEEC33FCEE9DECA7
:10081E00984005FCEE9DFE0FD5F0E9E4CEFD22EDED
:10082E00F8F5F0EE8420D21CFEADF075F008EF2F37
:10083E00FFED33FD4007985006D5F0F222C398FD28
:05084E000FD5F0EA22C5
:10085300C2D5EC30E709B2D5E4C39DFDE49CFCEEC0
:1008630030E715B2D5E4C39FFFE49EFE1207FEC333
:10087300E49DFDE49CFC80031207FE30D507C3E42E
:060883009FFFE49EFE222F
:10002600E56B245FF8E6056B22785C300702785FA3
:10003600E475F0011208F40207D32000EB7F2ED2FC
:10004600008018EF540F2490D43440D4FF30040BB2
:10005600EF24BFB41A0050032461FFE56C6002155B
:100066006C056FE56F7002056E30070D785CE47500
:10007600F0011208F4EF0208E2020D4B7403D207F6
:100086008003E4C207F56B8B5C8A5D895EE4F56CE0
:10009600F56EF56FE56C60077F2012006180F575DF
:1000A6006DFFC201C200C202C203C205C206C20877
:1000B60012002FFF700D3007057F00120072AF6F20
:1000C600AE6E22B4255FC2D5C20412002FFF24D023
:1000D600B40A00501A75F00A786C30D50508B6FFD8
:1000E6000106C6A426F620D5047002D20380D924C0
:1000F600CFB41A00EF5004C2E5D204020272D20154
:1001060080C6D20080C0D20280BCD2D580BAD205C9
:1001160080B47F201200612002077401B56C004094
:10012600F1120026FF12006102009AD208D2068060
:1001360095120026FB120026FA120026F94A4B7089
:100146000679437A037BFF20022EE56C602A7E0047
:100156008E827583001208B560060EEE656D70F02E
:10016600C2D5EBC0E0EAC0E0E9C0E0EE1202B9D0C9
:10017600E0F9D0E0FAD0E0FB1207D3FF60AAEBC0AB
:10018600E0EAC0E0E9C0E0120061D0E02401F9D065
:10019600E03400FAD0E0FBE56D0460DCD56DD98073
:1001A600877BFF7A0279B5D202809C79108002792A
:1001B60008C206C2088008D2D5790A8004790AC224
:1001C600D5E56D047002F56DE4FAFDFEFF1200261A
:1001D600FC7B08200113120026FD7B1030000A125A
:1001E6000026FE120026FF7B20EC3382D592D550E6
:1001F60013C3E43000069FFFE49EFEE42001039D46
:10020600FDE49CFCE4CBF8C201EC700CCFCECDCC67
:10021600E824F8F870F38017C3EF33FFEE33FEEDF2
:1002260033FDEC33FCEB33FB994002FB0FD8E9EBD3
:10023600300105F8D0E0C448B201C0E00AEC4D4EEA
:100246004F78207B0070C2EAB56D0040BCC0E0125A
:1002560002BBD0F0D0E0200104C4C0E0C4B201C0AB
:10026600F012004AD0F0D5F0EB02009A1209040110
:10027600375301B15801084C01044201B54F01BD85
:0F0286004401BD49011D4301C35501A74601A70E
:100295004501A747036350010C2D01102E01332B97
:1002A500011423013120034C2A00CC480000012B06
:1002B5003F3F3F00790AA2D5200314300509B91044
:1002C500020404B9080104A2D52006025001042045
:1002D50002689202B56C005034C0E07F20300319EB
:1002E5007F30A20272067205500F120312C202C2BB
:1002F50006C205C2087F30800F300503E9C0E01251
:100305000061300503D0E0F9D0E0B56CCC300517BD
:100315007F30B9100C1200617F583004077F788058
:1003250003B908031200613002057F2D0200617FC9
:10033500202008F87F2B2006F322920280CF286E1A
:10034500756C6C2900D2011200263001F8C20178C3
:100355006C30D50108F60200CC2D504349581200E7
:10036500262403B405004001E490035E9312005275
:0D037500743A120052D203756C040201B1FB
:100A66008B5C8A5D895EAB5FAA60A9611207D36061
:100A760063AB5CAA5DA95E1207D3605F855F628582
:100A860060638561648B658A668967AB62AA63A9C0
:100A9600641207D3FF6023AB65AA66A9671207D362
:100AA6006F7017042564F564E43563F563740125F6
:100AB60067F567E43566F56680D1AB62AA63A9641B
:100AC6001207D37002800D7401255EF55EE4355D74
:100AD600F55D809DAB5CAA5DA95E227B007A0079FC
:020AE6000022EC
:10088900EF4E6012EF60010EEDBB010B89828A8386
:10089900F0A3DFFCDEFA2289F05007F709DFFCA993
:0C08A900F022BBFEFCF309DFFCA9F022EA
:1009E600020E1AE493A3F8E493A34003F68001F2FF
:1009F60008DFF48029E493A3F85407240CC8C33312
:100A0600C4540F4420C8834004F456800146F6DFE0
:100A1600E4800B0102040810204080900CC8E47E9C
:100A2600019360BCA3FF543F30E509541FFEE493D5
:100A3600A360010ECF54C025E060A840B8E493A39C
:100A4600FAE493A3F8E493A3C8C582C8CAC583CAC7
:100A5600F0A3C8C582C8CAC583CADFE9DEE780BE7F
:010CF90000FA
:1008B500BB010CE58229F582E5833AF583E02250F8
:1008C50006E92582F8E622BBFE06E92582F8E22242
:0D08D500E58229F582E5833AF583E493225C
:1008E200BB010689828A83F0225002F722BBFE01F5
:0208F200F322EF
:1008F400FAE6FB0808E6F925F0F618E6CA3AF62205
:10090400D083D082F8E4937012740193700DA3A382
:1009140093F8740193F5828883E473740293686096
:06092400EFA3A3A380DF96
:100D4B00EFB40A07740D120D56740A309811A89956
:100D5B00B8130CC2983098FDA899C298B811F63008
:070D6B0099FDC299F59922E0
:00000001FF
